:020000040800F2
:1000000000070020F5040008FD2A0008B52A0008B2
:10001000DD2A0008B52A0008D52A0008F7040008E0
:10002000F7040008F7040008F7040008F13A000894
:10003000F7040008F7040008F7040008F7040008B4
:10004000F7040008F7040008F7040008F7040008A4
:10005000F7040008F7040008254F00084D4F00087A
:10006000754F00089D4F0008C54F0008F7040008B1
:10007000F7040008F7040008F7040008F704000874
:10008000F7040008F7040008F7040008692A0008CC
:10009000952A0008A52A0008F7040008ED4F00087B
:1000A000F7040008F7040008F7040008F704000844
:1000B000F7040008F7040008F7040008F704000834
:1000C000F7040008F7040008F7040008F704000824
:1000D000F7040008C1500008D5500008F7040008D4
:1000E00051500008F7040008F7040008F70400085E
:1000F000F7040008F7040008F7040008F7040008F4
:10010000F7040008F7040008E9500008F7040008A5
:10011000F7040008F7040008F7040008F7040008D3
:10012000F7040008F7040008F7040008F7040008C3
:10013000F7040008F7040008F7040008F7040008B3
:10014000F7040008F7040008F7040008F7040008A3
:10015000F7040008F7040008F7040008F704000893
:10016000F7040008F7040008F7040008F704000883
:10017000F7040008F7040008F7040008F704000873
:10018000F7040008F7040008F7040008F704000863
:10019000F7040008F7040008F7040008F704000853
:1001A000F7040008F7040008F7040008F704000843
:1001B000F7040008F7040008F7040008F704000833
:1001C000F7040008F7040008F7040008F704000823
:1001D000F7040008F7040008F7040008F704000813
:1001E000D916000800000000000000000000000018
:1001F00053B94AB9002908BF00281CBF4FF0FF318E
:100200004FF0FF3000F074B9ADF1080C6DE904CE89
:1002100000F006F8DDF804E0DDE9022304B07047E1
:100220002DE9F047089D04468E46002B4DD18A42A9
:10023000944669D9B2FA82F252B101FA02F3C2F1DC
:10024000200120FA01F10CFA02FC41EA030E94406D
:100250004FEA1C48210CBEFBF8F61FFA8CF708FB8E
:1002600016E341EA034306FB07F199420AD91CEB66
:10027000030306F1FF3080F01F81994240F21C8198
:10028000023E63445B1AA4B2B3FBF8F008FB1033E0
:1002900044EA034400FB07F7A7420AD91CEB040415
:1002A00000F1FF3380F00A81A74240F207816444E5
:1002B000023840EA0640E41B00261DB1D44000236A
:1002C000C5E900433146BDE8F0878B4209D9002DCE
:1002D00000F0EF800026C5E9000130463146BDE858
:1002E000F087B3FA83F6002E4AD18B4202D38242C2
:1002F00000F2F980841A61EB030301209E46002D71
:10030000E0D0C5E9004EDDE702B9FFDEB2FA82F2C5
:10031000002A40F09280A1EB0C014FEA1C471FFA23
:100320008CFE0126200CB1FBF7F307FB131140EA0A
:1003300001410EFB03F0884208D91CEB010103F1D7
:10034000FF3802D2884200F2CB804346091AA4B299
:10035000B1FBF7F007FB101144EA01440EFB00FE6D
:10036000A64508D91CEB040400F1FF3102D2A645D2
:1003700000F2BB800846A4EB0E0440EA03409CE771
:10038000C6F12007B34022FA07FC4CEA030C20FA1E
:1003900007F401FA06F31C43F9404FEA1C4900FA3E
:1003A00006F3B1FBF9F8200C1FFA8CFE09FB1811BB
:1003B00040EA014108FB0EF0884202FA06F20BD92E
:1003C0001CEB010108F1FF3A80F08880884240F27E
:1003D0008580A8F102086144091AA4B2B1FBF9F0C2
:1003E00009FB101144EA014100FB0EFE8E4508D9BD
:1003F0001CEB010100F1FF346CD28E456AD9023842
:10040000614440EA0840A0FB0294A1EB0E01A14226
:10041000C846A64656D353D05DB1B3EB080261EB94
:100420000E0101FA07F722FA06F3F1401F43C5E96E
:10043000007100263146BDE8F087C2F12003D840A4
:100440000CFA02FC21FA03F3914001434FEA1C47E6
:100450001FFA8CFEB3FBF7F007FB10360B0C43EAD8
:10046000064300FB0EF69E4204FA02F408D91CEB88
:10047000030300F1FF382FD29E422DD90238634486
:100480009B1B89B2B3FBF7F607FB163341EA034126
:1004900006FB0EF38B4208D91CEB010106F1FF3875
:1004A00016D28B4214D9023E6144C91A46EA00466C
:1004B00038E72E46284605E70646E3E61846F8E6FE
:1004C0004B45A9D2B9EB020864EB0C0E0138A3E747
:1004D0004646EAE7204694E74046D1E7D0467BE728
:1004E000023B614432E7304609E76444023842E7A0
:1004F000704700BF02E000F000F8FEE772B6374830
:1005000080F30888364880F3098836483649086001
:1005100040F20000CCF200004EF63471CEF2000141
:100520000860BFF34F8FBFF36F8F40F20000C0F23F
:10053000F0004EF68851CEF200010860BFF34F8FF5
:10054000BFF36F8F4FF00000E1EE100A4EF63C71E2
:10055000CEF200010860062080F31488BFF36F8F8D
:1005600004F0E2FA04F07AFB4FF055301F491B4AC1
:1005700091423CBF41F8040BFAE71D49184A9142E9
:100580003CBF41F8040BFAE71A491B4A1B4B9A423D
:100590003EBF51F8040B42F8040BF8E7002018495D
:1005A000184A91423CBF41F8040BFAE704F0C0FA44
:1005B00004F0A2FB144C154DAC4203DA54F8041BB2
:1005C0008847F9E700F042F8114C124DAC4203DACB
:1005D00054F8041B8847F9E704F0A8BA0007002084
:1005E000002300200000000808ED00E000010020CA
:1005F0000007002090550008002300208C230020D5
:1006000090230020284F0020E0010008E4010008AA
:10061000E4010008E40100082DE9F04F2DED108AF7
:10062000C1F80CD0C3689D46BDEC108ABDE8F08FC0
:10063000002383F311882846A047002003F0D4FE4E
:10064000FEE703F037FE00DFFEE70000F8B501F03B
:1006500055F804F003FA074604F052FA0546B8BB11
:10066000204B9F4234D001339F4234D01E4B27F0A1
:10067000FF029A4232D1F8B200F044FE2E4642F216
:10068000107400F045FE08B10024264601F02AFB54
:1006900020B1032000F07CF80024264635B1134B2E
:1006A0009F4203D004F024FA00242646002004F0E0
:1006B000DFF90EB100F082F801F0A4F900F086FE37
:1006C00001F088F8204600F0CDF800F077F8F9E75F
:1006D0002E460024D5E704460126D2E7064641F21D
:1006E0008834CEE7010007B0000008B0263A09B010
:1006F00008B501F03BF8A0F120035842584108BD6D
:1007000007B541F21203022101A8ADF8043001F04F
:100710004BF803B05DF804FB38B5302383F3118840
:10072000174803680BB103F01DFF164A1448002355
:100730004FF47A7103F00CFF002383F31188124CFD
:10074000236813B12368013B2360636813B16368B6
:10075000013B63600D4D2B7833B963687BB9022090
:1007600001F0E6F8322363602B78032B07D163682E
:100770002BB9022001F0DCF84FF47A73636038BDC6
:100780009023002019070008B0240020A82300208F
:10079000084B187003280CD8DFE800F008050208A1
:1007A000022001F0C3B8022001F0BEB8024B0022C3
:1007B0005A607047A8230020B024002010B501F033
:1007C00091FA30B1204B03221A70204B00225A605C
:1007D00010BD1F4B1F4A1C4619680131F8D0043365
:1007E0009342F9D162681C4B9A42F1D91B4B9B682A
:1007F00003F1006303F580339A42E9D204F04CF927
:1008000004F05EF9002000F0FFFF0220FFF7C0FFB8
:10081000134B1A6C00221A64196E1A66196E596C01
:100820005A64596E5A665B6E72B64FF0E0233021FF
:10083000C3F8084DD4E9003281F311889D4683F353
:1008400008881047C4E700BFA8230020B024002078
:100850000000010820000108FFFF0008002300201D
:10086000003802402DE9F04F93B0AC4B00902022AD
:10087000FF210AA89D6801F06FF8A94A1378A3B96F
:10088000A848012103601170302383F311880368A5
:100890000BB103F067FEA44AA24800234FF47A711B
:1008A00003F056FE002383F31188009B13B19F4B86
:1008B000009A1A609E4A009C1378032B1EBF0023E7
:1008C00013709A4A4FF0000A18BF5360D346564639
:1008D000D146012001F02AF824B1944B1B68002B6B
:1008E00000F01582002000F041FF0390039B002BD5
:1008F00001DA00F0B3FD039B002BEDDB012001F0DA
:1009000013F8039B213B162BE3D801A252F823F0E6
:100910006D09000895090008290A0008D308000895
:10092000D3080008D3080008B30A0008830C0008A5
:100930009D0B0008FF0B0008270C00084D0C000859
:10094000D30800085F0C0008D3080008D10C000889
:100950000D0A0008D3080008150D000879090008E1
:100960000D0A0008D3080008FF0B00080220FFF75B
:10097000BFFE002840F0F581009B0221BAF1000F74
:1009800008BF1C4605A841F21233ADF8143000F040
:100990000BFF9EE74FF47A7000F0E8FE071EEBDBDA
:1009A0000220FFF7A5FE0028E6D0013F052F00F248
:1009B000DA81DFE807F0030A0D10133605230593EB
:1009C000042105A800F0F0FE17E054480421F9E7DF
:1009D00058480421F6E758480421F3E74FF01C0873
:1009E000404600F013FF08F104080590042105A813
:1009F00000F0DAFEB8F12C0FF2D1012000FA07F76F
:100A000047EA0B0B5FFA8BFB4FF0000900F0F0FF99
:100A100026B10BF00B030B2B08BF0024FFF770FE71
:100A200057E746480421CDE7002EA5D00BF00B0375
:100A30000B2BA1D10220FFF75BFE074600289BD0BD
:100A4000012000F0E1FE0220FFF7A2FE00265FFA7F
:100A500086F8404600F0E8FE044690B1002140468A
:100A600000F0F2FE01360028F1D1BA46044641F208
:100A70001213022105A8ADF814303E4600F094FE92
:100A800027E70120FFF784FE2546244B9B68AB42F5
:100A900007D9284600F0BAFE013040F067810435DE
:100AA000F3E7234B00251D70204BBA465D603E46A0
:100AB000ACE7002E3FF460AF0BF00B030B2B7FF481
:100AC0005BAF0220FFF764FE322000F04FFEB0F172
:100AD0000008FFF651AF18F003077FF44DAF0F4A3F
:100AE000926808EB050393423FF646AFB8F5807F66
:100AF0003FF742AF124B0193B84523DD4FF47A70B4
:100B000000F034FE0390039A002AFFF635AF019BF4
:100B1000039A03F8012B0137EDE700BF0023002003
:100B2000AC2400209023002019070008B0240020E6
:100B3000A823002004230020082300200C230020E9
:100B4000AC230020C820FFF7D3FD074600283FF460
:100B500013AF1F2D11D8C5F1200242450AAB25F075
:100B6000030028BF424683490192184400F0E2FE88
:100B7000019A8048FF2100F0EFFE4FEAA8037D496B
:100B80000193C8F38702284600F0EEFE06460028CF
:100B90003FF46DAF019B05EB830537E70220FFF7BC
:100BA000A7FD00283FF4E8AE00F06EFE00283FF4F9
:100BB000E3AE0027B846704B9B68BB4218D91F2F85
:100BC00011D80A9B01330ED027F0030312AA134455
:100BD00053F8203C05934046042205A901F03AF859
:100BE00004378046E7E7384600F010FE0590F2E74C
:100BF000CDF81480042105A800F0D6FD06E70023F7
:100C0000642104A8049300F0C5FD00287FF4B4AE6D
:100C10000220FFF76DFD00283FF4AEAE049800F00F
:100C20001BFE0590E6E70023642104A8049300F06E
:100C3000B1FD00287FF4A0AE0220FFF759FD002887
:100C40003FF49AAE049800F017FEEAE70220FFF79F
:100C50004FFD00283FF490AE00F026FEE1E70220B1
:100C6000FFF746FD00283FF487AE05A9142000F0E9
:100C700021FE04210746049004A800F095FD3946A2
:100C8000B9E7322000F072FD071EFFF675AEBB0714
:100C90007FF472AE384A926807EB090393423FF63D
:100CA0006BAE0220FFF724FD00283FF465AE27F06D
:100CB00003074F44B9453FF4A9AE484600F0A6FDEE
:100CC0000421059005A800F06FFD09F10409F1E782
:100CD0004FF47A70FFF70CFD00283FF44DAE00F0A2
:100CE000D3FD002844D00A9B01330BD008220AA967
:100CF000002000F039FE00283AD02022FF210AA867
:100D000000F02AFEFFF7FCFC1C4803F073FB13B055
:100D1000BDE8F08F002E3FF42FAE0BF00B030B2B32
:100D20007FF42AAE0023642105A8059300F032FD6C
:100D3000074600287FF420AE0220FFF7D9FC80464A
:100D400000283FF419AEFFF7DBFC41F2883003F0D6
:100D500051FB059800F06AFE464600F049FE3C460D
:100D6000B7E5064652E64FF0000905E6BA467EE6CC
:100D700037467CE6AC23002000230020A08601003B
:100D8000094A136849F2690099B21B0C00FB013350
:100D90001360064B186844F2506182B2000C01FBEC
:100DA0000200186080B2704718230020142300202E
:100DB00010B500211022044600F0CEFD034B03CBFA
:100DC000206061601868A06010BD00BF107AFF1F2E
:100DD0002DE9F041ADF54E7D0DF134086CAC40F2DB
:100DE000751207460D460EA80021C8F8001000F045
:100DF000B3FD4FF4C4720021204600F0ADFD01F0B8
:100E000085FE254B4FF47A72B0FBF2F0186093E840
:100E10000700012384E807000DF5E9702382FFF73E
:100E2000C7FF4FF4A6431D49238406A804F072FAB5
:100E3000192384F832310DF2E32206AB0DF1300CA8
:100E40001E4603CE664510605160334602F108022B
:100E5000F6D13378137041460122204600F000FE9F
:100E600000230393AB7E029305F11903019380B233
:100E70000123CDE904800093E97E05A3D3E9002393
:100E8000384602F00BFA0DF54E7DBDE8F08100BF4B
:100E90009E6AC421818A46EEB824002024530008AB
:100EA0002DE9F043224DBBB001F030FEAB6840F2BB
:100EB000ED22C31A934232D906AFA8602B462822EE
:100EC0000021384602F09AFB05F10E0000F03CFDCF
:100ED000002604465FFA80F905F10E08F3B2F1002E
:100EE000994501F1280107D908EB06030822384685
:100EF00002F084FB0136F1E708230122CDE902323A
:100F000005340C4B0193A4B230230093CDE9047453
:100F100005A3D3E90023297B074802F0BFF93BB0C2
:100F2000BDE8F083AFF3008078F6339F93CACD8D90
:100F3000D0450020DD450020D0340020F0B58B8A5C
:100F4000013B9BB2C92BC9B006460C4647D8274D7A
:100F50002F7B27BB05F10C03009308223B46394643
:100F6000204602F00FFA7B1CFAB2D9001F46A38A72
:100F7000013B9A4205DA0E322A44009200230822ED
:100F8000EEE700230022C5E900230023AB6085F8CB
:100F9000D730C5F8D8302B7B0BB9E37E2B73812279
:100FA000002106AD27A800F0D7FC0122294627A87A
:100FB00000F024FE00230393A37E029304F119039F
:100FC00080B201932823CDE90450E17E009330469E
:100FD00004A3D3E9002302F061F9FFF761FF49B0F0
:100FE000F0BD00BF26417272DF25D7B7D045002083
:100FF00070B50D4614461E4602F0ACF850B9022EEC
:1010000010D1012C0ED112A3D3E90023C5E900238E
:10101000012007E0282C10D005D8012C09D0052C80
:101020000FD0002070BD302CFBD10BA3D3E90023DF
:10103000ECE70BA3D3E90023E8E70BA3D3E90023F4
:10104000E4E70BA3D3E90023E0E700BFAFF30080A0
:10105000401DA12026812A0B78F6339F93CACD8D9F
:101060009E6AC421818A46EE26417272DF25D7B777
:10107000F017304A39059E562DE9F04F8DB002AF7A
:1010800080460D4602F066F8044600285CD12B7EAF
:10109000022B1BD1EB8A012B18D101F037FD06463C
:1010A000FFF76EFE03464FF4C870DFF81C92B3FBE7
:1010B000F0F206F5167602FB103316FA83F3C9F840
:1010C0000030EB7E33B97B4B00221A702C37BD46C3
:1010D000BDE8F08FAB8AE6B2013BB34204F10104F4
:1010E0000CD907F108031E44E100009600230822F2
:1010F00001F0F801284602F045F9EBE707F1180086
:10110000FFF756FE324607F1180107F1080004F018
:101110008BF80028D7D10F2E08D8664B1E70D9F84F
:101120000030A3F51673C9F80030CFE7FB1DF87146
:101130000146009307220346284602F023F9F97975
:10114000404601F0FFFFC1E7EB8A282B26D010D8DC
:10115000012B1ED0052BB9D1BFF34F8F5649574BEA
:10116000CA6802F4E0621343CB60BFF34F8F00BF45
:10117000FDE7302BAAD16B7E514C0133627BDBB291
:101180009342E94603D1EA7E237B9A420BD0CD46B7
:101190009CE729464046FFF71BFE97E72946404655
:1011A000FFF7CCFE92E74FF0000807F11803A7F80D
:1011B00018801022009341460123284602F0E2F8ED
:1011C000AE8A023EB6B2F31C9B109B000733DB08CD
:1011D000A9EBC3039D460DF1080A1FFA88F34FEAF5
:1011E000C8019E4201F110010AD90AEB08030093DD
:1011F00008220023284602F0C5F808F10108ECE7B0
:1012000094F8D70000F010FBD4F8D810054619B9AF
:1012100094F8D70000F018FBD4F8D83033449D423E
:1012200005D294F8D7000021013000F00DFB4FEA01
:10123000960B4FF000081FFA88F18B45D4E9003275
:1012400009D90AEB880103EB8800012200F08CFB2E
:1012500008F10108EFE7F31842F10002C4E9003297
:10126000D4F8D83094F8D70006EB0308C4F8D88037
:1012700000F0DAFA804509D394F8D730D4F8D800D2
:101280000133401B84F8D730C4F8D800FF2E0D4D31
:1012900009D80023237300F0F7FA00F023FD28811A
:1012A00008B9FFF78BFA23689B0A01332B810023CF
:1012B000A3606CE7C934002000ED00E00400FA05EB
:1012C000D0450020B8240020CC34002010B50A4BB3
:1012D0000A4A1A6003F5805393F860203AB9DC6D2E
:1012E0002CB1204600F076FD204603F053FFBDE808
:1012F0001040034800F06EBD00350020DC530008AC
:1013000048450020014B1870704700BFC4240020DE
:1013100030B54FF00054244B22689A4285B007D074
:1013200003F0F8FB0446A8B90024204605B030BD00
:101330001E4B627D1A701E48237D03731D49C9220E
:101340000E3000F0F7FA2046E022002100F004FB06
:101350000124EAE7184A194D136C43F00073136433
:10136000AA6D174B9A42DFD12B6E013B7E2BDBD847
:10137000144A07CA01AB83E807001846032100F0AE
:101380007FFC6B6D83424FF00003CDD12A6D8A4202
:1013900001BFAB65054B2A6E1A7003BF0A4BEA6D9D
:1013A0001A601C46C1E700BF9AAD44C5C4240020A2
:1013B000D0450020160000200038024000660040A2
:1013C0005041A0B0586600401023002037B51A4D98
:1013D00000F088FC02236B71184B288119681848AB
:1013E000012201F031FA00230193164B16490093B4
:1013F0001648174B4FF4805201F07CFE154B1978BC
:1014000011B1124801F09EFE01F080FB0446FFF787
:10141000B7FC4FF4C873B0FBF3F202FB130304F5FF
:10142000167010FA83F00C4B186003F069FB08B1DA
:101430000F232B8103B030BDB824002010230020DF
:1014400000350020F10F0008C8240020D03400200F
:1014500079100008C4240020CC3400202DE9F04F7E
:101460002DED028B93A7D7E900670FF25029D9E938
:1014700000898A4C95B0DFF84CA2DFF84CB22046C8
:1014800001F038FF034650B30025CDE91155109502
:10149000ADF84C50027B8DF84C209968406811AA39
:1014A00003C21B6843F00043109301F031FB10EBC3
:1014B0000A0241F10003009510A9584600F0F2FD20
:1014C000A842774A05DD204601F018FF744A1570DE
:1014D000D5E71378072B00F2B980013313700DADF7
:1014E0009FED6C8B0023DFF8E0B10C93ADF83C303E
:1014F0000D936B6000230DF125028DED008B4FF0F5
:10150000010A09A958468DF825308DF824A001F06C
:101510004BF99DF824200023002A40F09B802046B0
:1015200001F018FE0546002847D1DFF8A0B101F010
:10153000EDFADBF8003098423FD301F0E7FA07906C
:10154000FFF71EFC079A4FF4C87302F51672B0FB42
:10155000F3F101FB130312FA83F3CBF80030DFF849
:1015600070B19BF800100791002914BF2B46534619
:1015700010A88DF83030FFF71BFC0799C1F110025D
:10158000D2B2062A10AB28BF062219440DF1310051
:10159000079200F0CFF9079A0CAB0393182302933C
:1015A0000132404BD2B2CDE900A304923B46324611
:1015B000204601F015FE8BF8005001F0A7FA3A4AD8
:1015C0003A4D1368C31AB3F57A7F32D3106001F035
:1015D0009FFA02460B46204601F09AFE204601F093
:1015E000B9FD30B32B7BDFF8ECA0002B14BF032335
:1015F00002238AF8053001F089FA0DF1400B4FF40F
:101600007A730122B0FBF3F05946CAF80000504645
:1016100000F0CCFA18230293254B019380B240F2DC
:101620005513CDE903B0009342464B46204601F0E6
:10163000D7FD2B7B2BB1FFF733FC2B7B002B7FF4EB
:101640001AAF15B0BDEC028BBDE8F08F204601F05B
:1016500055FE44E71946102210A800F07DF90DF15F
:1016600026030AAA0CA9584600F01AFE95E80300C2
:1016700011AB83E803009DF83C308DF84C300C9B97
:10168000109310A9DDE90A23204602F015F831E78E
:10169000AFF300800000000000000000D034002004
:1016A000B5460020C8340020B0460020D0450020B8
:1016B000B4460020401DA12026812A0BF1C6A7C1F7
:1016C000D068080F40420F0000350020CC340020C5
:1016D000C9340020B824002008B5054800F07AFE7F
:1016E000BDE80840034A0449002003F04DBD00BF97
:1016F0000035002004470020CD120008704700008C
:101700002DE9F84F4FF47A73DFF85880DFF85890DE
:1017100006460D4602FB03F7002498F900305A1CD8
:101720005FFA84FA01D0A34212D159F82400036869
:101730002A46D3F820B031463B46D847854207D1E8
:10174000074B012083F800A0BDE8F88F0124E4E7EF
:10175000002CFBD04FF4FA7002F04CFE0020F3E7AF
:10176000F84600201C2300202023002007B500237A
:10177000024601210DF107008DF80730FFF7C0FF89
:1017800020B19DF8070003B05DF804FB4FF0FF3077
:10179000F9E700000A4608B50421FFF7B1FF80F021
:1017A0000100C0B2404208BD30B4074B0A46197868
:1017B000064B53F821402368DD69054B0146AC46D2
:1017C000204630BC604700BFF846002020230020A0
:1017D000A086010070B502F0D1FF094E094D30809E
:1017E000002428683388834208D902F0C1FF2B689F
:1017F00004440133B4F5803F2B60F2D370BD00BFC9
:10180000FA460020B846002003F07AB800F10060E4
:1018100000F580300068704700F10060920000F52C
:10182000803002F0F9BF0000054B1A68054B1B8899
:101830009B1A834202D9104402F09ABF00207047DD
:10184000B8460020FA460020024B1B68184402F0FC
:10185000AFBF00BFB846002010F003030AD1B0F5B7
:10186000047F05D200F10050A0F51040D0F80038F8
:10187000184670470023FBE700F10050A0F5104028
:10188000D0F8100A70470000064991F8243033B1AF
:101890000023086A81F824300822FFF7BDBF012029
:1018A000704700BFBC460020014B1868704700BF5E
:1018B000002004E070B5194B1D68194B0138C5F3C1
:1018C0000B0408442D0C04221E88A6420BD15C6830
:1018D0000A46013C824213460FD214F9016F4EB101
:1018E00002F8016BF6E7013A03F10803ECD18142FB
:1018F0000B4602D22C2203F8012B0A4A0524168833
:10190000AE4204D1984284BF967803F8016B013C43
:1019100002F10402F3D1581A70BD00BF002004E0A8
:10192000805300086C5300087047000070470000A7
:101930007047000010B50023934203D0CC5CC45420
:101940000133F9E710BD000003460246D01A12F930
:10195000011B0029FAD1704702440346934202D08A
:1019600003F8011BFAE770472DE9F8431F4D1446B1
:1019700095F824200746884652BBDFF870909CB348
:1019800095F824302BB92022FF2148462F62FFF71B
:10199000E3FF95F82400C0F10802A24228BF2246C6
:1019A000D6B24146920005EB8000FFF7C3FF95F8E1
:1019B0002430A41B1E44F6B2082E17449044E4B20F
:1019C00085F82460DBD1FFF75FFF0028D7D108E05E
:1019D0002B6A03EB82038342CFD0FFF755FF002829
:1019E000CBD10020BDE8F8830120FBE7BC460020F6
:1019F000024B1A78024B1A70704700BFF84600205D
:101A00001C23002010B5074C074920684FF4E13330
:101A10000B6002F0B5FB60680349BDE8104002F0BE
:101A2000AFBB00BF20230020E4460020094B10B5C7
:101A30001422044600211846FFF78EFF064A074B82
:101A4000127804600146BDE8104053F8220002F00D
:101A500097BB00BFE4460020F8460020202300206A
:101A60002DE9F0470D46044600219046284640F2F5
:101A70007912FFF771FF234620220021284601F04A
:101A8000BDFD231D02222021284601F0B7FD631D64
:101A900003222221284601F0B1FDA31D03222521A6
:101AA000284601F0ABFD04F1080310222821284646
:101AB00001F0A4FD04F1100308223821284601F0AA
:101AC0009DFD04F1110308224021284601F096FDF6
:101AD00004F1120308224821284601F08FFD04F189
:101AE000140320225021284601F088FD04F1180338
:101AF00040227021284601F081FD04F120030822D4
:101B0000B021284601F07AFD04F121030822B82112
:101B1000284601F073FD04F12207C0263B463146FA
:101B200008222846083601F069FDB6F5A07F07F1C6
:101B30000107F3D104F1320308223146284601F0AF
:101B40005DFD002704F1330A94F832304FEAC709EB
:101B50009F4209F5A47615D3B8F1000F08D131469C
:101B600004F599730722284601F048FD09F24F1643
:101B7000274694F832213B1B93420CD3F01DC0083A
:101B8000BDE8F0870AEB070308223146284601F03A
:101B900035FD0137D8E707F23313314608222846CE
:101BA00001F02CFD08360137E3E7000013B50446C9
:101BB0000846002101602346C0F80310202201904E
:101BC00001F01CFD0198231D0222202101F016FDC9
:101BD0000198631D0322222101F010FD0198A31D2D
:101BE0000322252101F00AFD019804F108031022C7
:101BF000282101F003FD072002B010BDF8B50E4604
:101C000005461446002181223046FFF7A5FE2B46EB
:101C100008220021304601F0F1FC7CB96B1C072240
:101C20000821304601F0EAFC0F2401236A785F1C8A
:101C3000013B934204D3E01DC008F8BD0824F4E73B
:101C4000EB1921460822304601F0D8FC08343B4607
:101C5000ECE7000030B5094D0A4491420DD011F86F
:101C6000013B5840082340F30004013B2C4013F093
:101C7000FF0384EA5000F6D1EFE730BD2083B8EDD2
:101C8000F7B54FF0FF33DFF854C0DFF854E000EB56
:101C900081011A4688421CD050F8044B019401AFD0
:101CA000042417F8015B82EA05620825DB18164652
:101CB00005F1FF355241002EBCBF83EA0C0382EAD6
:101CC0000E0215F0FF05F1D1013C14F0FF04E8D13C
:101CD000E0E7D843D14303B0F0BD00BF9336EAA993
:101CE000EBE1F042F7B5354A106851686B4603C323
:101CF0006A4633493348082303F0A6FA044688BBF2
:101D00000A25314A106851686B4603C36A462F4959
:101D10002C48082303F098FA0446002845D00369AC
:101D2000B3F5702F41D8B0F86620532A3DD1284A28
:101D3000024402F15C018B4237D35C3B2149002015
:101D40009E1AFFF787FF3246074604F16401002020
:101D5000FFF780FFA3689F4227D1E368984208BF3E
:101D6000002522E00369B3F5702F25D8428B532A52
:101D700020D1174A024402F110018B4218D3103BC4
:101D8000104900209D1AFFF765FF2A46064604F118
:101D900018010020FFF75EFFA3689E4202D1E368AE
:101DA000984201D00D25ACE70025284603B0F0BDD0
:101DB0001025A6E70C25A4E70B25A2E7A0530008F1
:101DC000DCFF0E0000000108A953000890FF0E0080
:101DD0000800FFF710B5037C044613B9006803F050
:101DE0001BFA204610BD00000023BFF35B8FC360C9
:101DF000BFF35B8FBFF35B8F8360BFF35B8F704775
:101E0000BFF35B8F0068BFF35B8F704770B505460B
:101E10000C30FFF7F5FF05F1080604463046FFF7E2
:101E2000EFFFA04206D930466D68FFF7E9FF254471
:101E3000281A70BD3046FFF7E3FF201AF9E70000CB
:101E400070B50546406898B105F10800FFF7D8FF66
:101E500005F10C0604463046FFF7D2FF84423046B7
:101E600094BF6D680025FFF7CBFF013C2C44201A7E
:101E700070BD000038B50C460546FFF7C7FFA0420D
:101E800010D305F10800FFF7BBFF04446868B4FBFA
:101E9000F0F100FB1144BFF35B8F0120AC60BFF396
:101EA0005B8F38BD0020FCE72DE9F0411446074662
:101EB0000D46FFF7C5FF844228BF0446D4B1B8469B
:101EC00058F80C6B4046FFF79BFF304428604046B3
:101ED0007E68FFF795FF331A9C4203D86C6001209F
:101EE000BDE8F0816B60A41B3B68AB602044E860F8
:101EF0000220F5E72046F3E738B50C460546FFF724
:101F00009FFFA04210D305F10C00FFF779FF0444B6
:101F10006868B4FBF0F100FB1144BFF35B8F012054
:101F2000EC60BFF35B8F38BD0020FCE72DE9FF417B
:101F3000884669460746FFF7B7FF6C4606B204EBD2
:101F4000C6060025B44209D06268206808EB050186
:101F5000FFF7F0FC636808341D44F3E72946384670
:101F6000FFF7CAFF284604B0BDE8F081F8B5054682
:101F70000C300F46FFF744FF05F1080604463046D3
:101F8000FFF73EFFA042304688BF6C68FFF738FF7E
:101F9000201A386020B130462C68FFF731FF20440A
:101FA000F8BD000073B5144606460D46FFF72EFF38
:101FB000844228BF04460190DCB101A93046FFF7F6
:101FC000D5FF019B33B93268C5E90233C5E9002466
:101FD00001200CE09C4238BF0194286001986860A1
:101FE0008442F5D93368AB60241AEC60022002B059
:101FF00070BD2046FBE700002DE9FF410F46694612
:10200000FFF7D0FF6C4600B204EBC0050026AC42DF
:1020100009D0D4F8048054F8081BB8194246FFF7D9
:1020200089FC4644F3E7304604B0BDE8F081000087
:1020300038B50546FFF7E0FF044601462846FFF79E
:1020400019FF204638BD0000302383F3118862B6A3
:1020500070470000002383F3118862B670470000C8
:1020600010B4026854681A4623465DF8044B1847BA
:102070000120704700207047002070477047000023
:10208000002070470E20704700F5805090F8C8007F
:10209000C0F340007047000000F5805090F9C9007F
:1020A00070470000F7B50C68BDF8207014F00054BC
:1020B0001E466FD10B7B082B6CD8FFF7C5FF456917
:1020C000AB685B010CD4AB681B0108D4AC6814F09E
:1020D00080545DD1FFF7BEFF204603B0F0BD012460
:1020E0000B6804F1180C002BB8BFDB004FEA0C1C86
:1020F000B4BF43F004035B0545F80C300B680FFADE
:1021000084FC13F0804F18BF05EB0C1E05EB0C1C74
:102110001EBFDEF8803143F00203CEF880310B7B26
:10212000CCF8843105EB04158B68C5F88C314B680D
:10213000C5F88831DCF8803143F00103CCF88031F8
:1021400000EB441541F268031D4403EB44130344C0
:10215000C5E9002608330D4601F10C0C55F804EBD7
:1021600043F804EB6545F9D184342D881D8000EBDC
:10217000441407F00303257925F00B052B43237145
:10218000FFF768FF0097334600F0E2FC0120A4E768
:102190000224A5E74FF0FF309FE7000013B500F5DC
:1021A00080540191E06DFFF74BFE1F280AD9019979
:1021B000E06D2022FFF7BAFEA0F1200358425841FB
:1021C00002B010BD0020FBE708B500F58050FFF716
:1021D0003BFFC06DFFF708FEBDE80840FFF73ABFC0
:1021E00000220260828142608260704710B5002246
:1021F0000023C0E900230023044603810C30FFF7CD
:10220000EFFF204610BD0000F0B5054600F58050F8
:102210000C4690F8C83013F0040FC3F3800108BFD8
:10222000114661F3820304F1840680F8C83005EB9F
:10223000461389B01B79D8072ED57AB319072DD448
:102240006846FFF7D3FF05EB441303F5835303F10F
:10225000180703AA103318685968144603C40833D2
:10226000BB422246F7D1186820609B88A380DDE935
:102270000E23CDE900230123ADF808302B68694611
:10228000DB6B2846984705EB46152B791A075CBF90
:1022900043F008032B7101E0002AF4D109B0F0BD2E
:1022A0002DE9F047074688B007F5805468469A46FE
:1022B0008846FFF7C9FE9146FFF798FFE06DFFF7EC
:1022C000A5FD1F2829D9E06D20226946FFF7B0FE41
:1022D000202822D103AD444605AB2E4603CE9E42B4
:1022E00020606160354604F10804F6D13068206052
:1022F000B388A380DDE90023C9E90023BDF80830D5
:10230000AAF80030FFF7A6FE4A4653464146384633
:1023100008B0BDE8F04700F009BCFFF79BFE0020C5
:1023200008B0BDE8F08700002DE9F84F0023C0E9B0
:102330000133254B044640F8183B0F46FFF750FF8A
:1023400004F12800FFF752FF04F1480804F5825514
:102350004646083530462036FFF748FFAE42F9D1F1
:1023600004F580554FF480534FF00009C5E9133947
:10237000C5F848800123EE6504F5875804F58456B6
:10238000C5F8549085F8583085F86030083608F163
:1023900008084FF0000A4FF0000B46E908ABA6F121
:1023A0001800FFF71DFF203646F8289C4645F4D15B
:1023B00085F8C97017B1054800F0A2FB044B6361B2
:1023C0002046BDE8F88F00BFDC530008B453000876
:1023D0000064004010B5044B197804464A1C1A707A
:1023E000FFF7A2FF204610BD004700202DE9F0476F
:1023F000002950D0294B2A4FB7FBF1F599428CBFE9
:102400000A231123581EB5FBF3FC03FB1C53C4B273
:102410002BB102280346F5D80020BDE8F0870CF167
:10242000FF36B6F5806FF7D2C4EBC40E0EF103038E
:102430004FEAE309C3F3C703A4EB030809F1010A58
:102440004FF47A755FFA88F009FB05555AFA88F857
:10245000B5FBF8F5B5F5617FC1BF0EF1FF33C3F3EE
:10246000C703E01AC0B25C1C50FA84F40CFB04F4FD
:10247000B7FBF4F4A142CFD1013BDBB20F2BCBD899
:102480000138C0B20728C7D800211071168091709A
:10249000D3700120C1E70846BFE700BF3F420F00ED
:1024A00040787D0170B505460E464FF47A746B692D
:1024B0005B6803F00103B34207D04FF47A7001F078
:1024C00099FF013CF3D1204670BD0120FCE70000DC
:1024D00030B54269936913F0700F16D000230B4C8E
:1024E000936103F1840200EB421211794D0709D583
:1024F000890707D5416954F823508D60117941F05F
:10250000040111710133032BEBD130BDC853000816
:1025100073B51D46436916469A68D207044609D525
:102520009A6801219960C2F34002CDE9006500215B
:10253000FFF76AFE63699A68D1050BD59A684FF474
:1025400080719960C2F34022CDE9006501212046E7
:10255000FFF75AFE63699A68D2030BD59A684FF465
:1025600080319960C2F34042CDE9006502212046E6
:10257000FFF74AFE204602B0BDE87040FFF7A8BF53
:10258000F8B50446466900296CD106F10C07386895
:1025900080076AD006EB01153868D5F8B00110F055
:1025A000040FD5F8B0011ABFC00840F00040400D3C
:1025B000A061D5F8B0C11CF0020F1CBF40F08040F4
:1025C000A061D5F8B40106EB011100F00F0084F80A
:1025D0002400D1F8B8012077D1F8B801000A60775B
:1025E000D1F8B801000CA077D1F8B801000EE0775F
:1025F000D1F8BC0184F82000D1F8BC01000A84F8AD
:102600002100D1F8BC01000C84F82200D1F8BC11E3
:10261000090E84F823103821396004F1340004F1E4
:10262000180104F1240551F8046B40F8046BA94229
:10263000F9D109880180C4E90A23214600232386B1
:1026400051F8283B2046DB6B984704F58052204622
:1026500092F8C83043F0040382F8C830BDE8F8406F
:10266000FFF736BF06F1100791E7F8BD10B5044635
:1026700000F04EFA02460B4652EA030102D0013A3C
:1026800063F100030449086820B12146BDE8104009
:10269000FFF776BF10BD00BFFC460020F8B500F57F
:1026A00083511E46FFF7D0FCDFF844C008310024F8
:1026B00004F1840500EB45152B795F070ED4DB068A
:1026C0000CD5D1E900739742B34107D243695CF856
:1026D00024709F602B7943F004032B710134032C89
:1026E00001F12001E4D1BDE8F840FFF7B3BC00BF21
:1026F000C853000808B5FFF7A7FCFFF7E9FEBDE8DF
:102700000840FFF7A7BC0000F8B543690546986884
:1027100000F0E050B0F1E05F0F461FD0E8B1FFF7E6
:1027200093FC05F583541034002606F1840305EB71
:1027300043131B791A0706D50136032E04F1200432
:10274000F3D1012007E05B07F6D42146384600F0BC
:1027500039FA0028F0D1FFF77DFCF8BD0120FCE735
:1027600000F5805008B5FFF76FFCC06DFFF74EFB1A
:10277000FFF770FC43090CBF0120002008BD0000DA
:10278000F8B51D46002313700F4606461446FFF7A2
:10279000E7FF80F00100387025B129463046FFF789
:1027A000B3FF2070F8BD00002DE9B8410C46154676
:1027B0001F46804600F0ACF90B462178024609B965
:1027C000287850B14046FFF769FFFFF793FF3B467B
:1027D0002A462146FFF7D4FF0120BDE8B88100005A
:1027E00010B5FFF731FC174B1A6C42F000721A64F7
:1027F0001A6A42F000721A621A6A00F5805422F0D6
:1028000000721A62FFF726FC94F8C830DB0718D470
:10281000B9B103211320FFF717FC01F0E5FA0321FA
:10282000142001F0E1FA0321152001F0DDFA94F8FB
:10283000C83043F0010384F8C830BDE81040FFF70A
:1028400009BC10BD003802402DE9F04700F5805565
:1028500088B095F8C930012B0446884616467FD8C3
:10286000804F57F823200AB947F82300D7F800A073
:10287000C4F80C802674BAF1000F63D095F8C93003
:10288000012B6FD001212046FFF7AAFFFFF7DCFBE9
:102890006269136823F0020313606269136843F0EE
:1028A00001031360636900275F6101212046FFF780
:1028B000D1FBFFF7F7FD002800F09580E86DFFF7EA
:1028C00093FA04F58359BA4609F108092022002138
:1028D0006846FFF741F802A8FFF782FCCDF818A080
:1028E0006A4609EB07030DF1180E9446BCE8030095
:1028F000F44518605960624603F10803F5D1DCF82D
:102900000000186020379CF804201A71602FDDD178
:1029100095F8C8306FF38203002785F8C8306A46FF
:1029200041462046ADF80070ADF802708DF8047095
:10293000FFF75CFD636948BB4FF400421A6008B0C2
:10294000BDE8F08741F2D00002F026FC814610B1CC
:102950005146FFF7E9FCC7F80090B9F1000F8DD19F
:102960000020ECE7386803681B6B98470146002895
:1029700088D13868FFF734FF3868036832465B68EF
:102980004146984700287FF47DAFE9E761221A604D
:102990009DF802309DF803201B06120402F47022F9
:1029A00003F040731343BDF80020C2F30902134340
:1029B0009DF804201205022E02F4E0020CBF4FF035
:1029C00000410021134362690B43D3616369132201
:1029D0005A616269136823F0010313603946204687
:1029E000FFF760FD08B96369A6E795F8C93093BBA6
:1029F0006169D1F8002242F00102C1F80022616948
:102A0000D1F8002222F47C5222F00E02C1F80022FA
:102A10006169D1F8002242F46062C1F80022626963
:102A2000C2F814326269C2F80432626941F6FF7179
:102A3000C2F80C126269C2F840326269C2F84432CC
:102A400063690122C3F81C226269D2F8003223F0C4
:102A50000103C2F8003295F8C83043F0020385F84C
:102A6000C8306CE7FC46002008B500F051F850EA89
:102A70000103024602D0421E61F10001044B1868B6
:102A800010B10B46FFF744FDBDE8084001F064B803
:102A9000FC46002008B50020FFF7E8FDBDE808402F
:102AA00001F05AB808B50120FFF7E0FDBDE8084085
:102AB00001F052B800B59BB0EFF309816822684677
:102AC000FEF738FFEFF30583014B9B6BFEE700BF7A
:102AD00000ED00E008B5FFF7EDFF000000B59BB08A
:102AE000EFF3098168226846FEF724FFEFF30583C0
:102AF000014B5B6BFEE700BF00ED00E0FEE700006E
:102B00000FB408B5029801F00BFCFEE701F044BFDA
:102B100001F01CBF13B56C4684E80600031D94E861
:102B2000030083E80500012002B010BD73B585687D
:102B3000019155B11B885B0707D4D0E900369B6B28
:102B40009847019AC1B23046A847012002B070BD33
:102B5000F0B5866889B005460C465EB1BDF83830E0
:102B60005B070AD4D0E900379B6B98472246C1B275
:102B70003846B047012009B0F0BD00220023CDE95E
:102B800000230023ADF808300A4603AB01F1080624
:102B9000106851681C4603C40832B2422346F7D17C
:102BA000106820609288A280FFF7B2FF0423ADF87E
:102BB00008302B68CDE90001DB6B69462846984751
:102BC000D8E7000030B503680968DD0FB5EBD17FA9
:102BD00023F0604421F060424FEAD1700BD0002B0B
:102BE000B8BFA40C0029B8BF920C944202D034BFE5
:102BF0000120002030BD944205D1C1F38070C3F3A1
:102C000080738342F6D194422CBF00200120F1E76B
:102C10002DE9F041456A15B94162BDE8F0814B6884
:102C200023F06047C3F38A464FEAD37EC3F380782C
:102C300016EA230638BF3E46AC462B465A68BEEB22
:102C4000D27F22F060440AD0002A18DAA40CB442E1
:102C500017D19D420FD10D60DEE71346EEE7A74284
:102C600007D102F08044C2F3807242450BD054B1C8
:102C7000EFE708D2EDE7CCF800100B60CDE7B442E7
:102C800001D0B442E5D81A689C46002AE5D1196003
:102C9000C3E700002DE9F047089D01F007044FEA63
:102CA000D508224405F0070500EBD1004FF47F4919
:102CB000944201D1BDE8F08704F0070705F0070A48
:102CC00057453E4638BF5646C6F10806111B8E4290
:102CD00028BF0E46E10808EBD50E415C13F80EC084
:102CE000B94029FA06F721FA0AF1FFB28CEA01018C
:102CF00047FA0AF739408CEA010C03F80EC0344455
:102D00003544D5E780EA0120082341F2210201B2CF
:102D10004000002980B203F1FF33B8BF504013F0E8
:102D2000FF03F4D17047000038B50C468D18A5425A
:102D300000D138BD14F8011BFFF7E4FFF7E70000EE
:102D400042684AB1136843604389818901339BB269
:102D50009942438138BF83811046704770B588B06F
:102D6000202204460D4668460021FEF7F5FD204668
:102D70000495FFF7E5FF024658B16B46054608AEDD
:102D80001C4603CCB44228606960234605F108055F
:102D9000F6D1104608B070BD082817D909280CD004
:102DA0000A280CD00B280CD00C280CD00D280CD0E5
:102DB0000E2814BF4020302070470C207047102090
:102DC000704714207047182070472020704700007B
:102DD000082817D90C280CD910280CD914280CD97C
:102DE00018280CD920280CD930288CBF0F200E2091
:102DF0007047092070470A2070470B2070470C204D
:102E000070470D20704700002DE9F843078C072F0D
:102E100004461ED9D0E9029800254FF6FF73C5F18C
:102E20002006A5F1200029FA05F108FA06F628FA8D
:102E300000F031430143C9B21846FFF763FF08357C
:102E4000402D0346EBD1E1693A46BDE8F843FFF770
:102E50006BBF4FF6FF70BDE8F883000010B54B68FC
:102E600023B9CA8A63F30902CA8210BD04691A68C9
:102E70001C600361C38A013BC3824A60EFE7000024
:102E80002DE9F84F1D46CB8A0F46C3F309010529EA
:102E9000814692460B4630D00020AAB207F11A04B0
:102EA0009EB2042E1FFA80F80FD8904503F101035B
:102EB00006D3FB8A0A4462F30903FB8201201AE06D
:102EC0001AF80060E6540130EAE79045F1D2A1F12A
:102ED000050B1C237C68BBFBF3F203FB12BB1FFA40
:102EE0008BF6002C45D14846FFF72AFF044638B937
:102EF00078606FF00200BDE8F88F4FF00008E6E759
:102F0000002606607860ADB24FF0000B454510D941
:102F10000AEB0803221D13F8011B9155B1B208F109
:102F200001081B291FFA88F82BD0454506F1010638
:102F3000F1D8FB8AC3F30902154465F30903BCE722
:102F4000013292B21C462368002BF9D16B1F0B444F
:102F50001C21B3FBF1F301339BB29A42D3D2BBF1F4
:102F6000000FD0D14846FFF7EBFE20B9C4F800B0FF
:102F7000BFE70122E7E7C0F800B05E4620600446E4
:102F8000C1E74545D5D94846FFF7DAFE08B92060C4
:102F9000AFE7C0F800B0002620600446B6E70000A6
:102FA0002DE9F04F2DED028B1C4683B05B69019239
:102FB00007468846002B00F09A80238C2BB1E269EB
:102FC000002A00F09480072B35D807F10C00FFF79A
:102FD000B7FE054638B96FF00205284603B0BDECD0
:102FE000028BBDE8F08F14220021FEF7B5FC228C85
:102FF000E16905F10800FEF79DFC208C013080B2EC
:10300000FFF7E6FEFFF7C8FE013880B220840130EA
:1030100028746369228C1B782A4403F01F0363F031
:103020003F0348F000411372384669602946FFF7B4
:10303000EFFD0125D1E700F10C034FF0000908EE88
:10304000103A4FF0800A4E464D4618EE100AFFF730
:1030500077FE83460028BED014220021FEF77CFCB8
:10306000002E3AD1019BABF8083002220BF1080E7A
:103070001FFA82FC0CF10100BCF1060F218C80B21A
:1030800001D88E422BD3FFF7A3FEFFF785FE6269BE
:103090001278013802F01F028E4208BF4FF0400A3A
:1030A00042EA49121BFA80F14AEA020A013048F06A
:1030B000004281F808A08BF81000CBF80420594694
:1030C0003846FFF7A5FD238C0135B3422DB289F0B8
:1030D00001094FF0000AB8D17FE70022C6E7E16995
:1030E000895D0EF802100136B6B20132C0E76FF00A
:1030F000010572E7F8B515460E4630220021044658
:103100001F46FEF729FC069B6360B5F5001F079B71
:10311000A76034BF6A094FF6FF72A36297B2E661F7
:1031200004F1100000239A4206D800230360A7820E
:10313000E3822383E360F8BD066001333046203626
:10314000F1E7000003781BB94BB2002BC8BF017038
:103150007047000000787047F8B50C46C96907460B
:1031600011B9238C002B37D1257E1F2D34D8387808
:1031700028BB228C072A2CD8268A36F003032BD1B1
:103180004FF6FF70FFF7D0FD20F001003102400440
:1031900041EA0561400C41EA40254FF6FF722346A3
:1031A00029463846FFF7FCFE002807DD62691378E0
:1031B0000133DBB21F2B88BF00231370F8BD218AB7
:1031C0002D0645EA012505432046FFF71DFE024670
:1031D000E5E76FF00300F1E76FF00100EEE70000B4
:1031E00070B58AB0044616460021282268461D465E
:1031F000FEF7B2FBBDF83830ADF810300F9B0593E9
:103200009DF840308DF81830119B07936946BDF842
:103210004830ADF820302046CDE90265FFF79CFF2D
:103220000AB070BD2DE9F041D36905460C4616463B
:103230000BB9138C5BBB377E1F2F28D895F8008005
:10324000B8F1000F26D03046FFF7DEFD33782102BB
:1032500041EAC33141EA0801338A41EA076141EAA0
:1032600003410246334641F080012846FFF798FEAD
:1032700000280ADD3378012B07D1726913780133F6
:10328000DBB21F2B88BF00231370BDE8F0816FF005
:103290000100FAE76FF00300F7E70000F0B58BB02C
:1032A00004460D4617460021282268461E46FEF7B2
:1032B00053FB9DF84C305A1E534253418DF8003059
:1032C0009DF84030ADF81030119B05939DF84830C3
:1032D0008DF81830149B07936A46BDF85430ADF84A
:1032E000203029462046CDE90276FFF79BFF0BB040
:1032F000F0BD0000406A00B104307047436A1A68AC
:10330000426202691A600361C38A013BC38270474B
:103310002DE9F041D0F82080194E14461D46414653
:10332000002709B9BDE8F081D1E90223A21A65EBB3
:103330000303964277EB03031ED2036A8B420DD13F
:10334000FFF78CFD036A1B68036203690B60C38A85
:103350000161016A013BC3828846E2E7FFF77EFD17
:103360000B68C8F8003003690B60C38A0161013B38
:10337000C382D8F80010D4E788460968D1E700BFB7
:1033800080841E002DE9F04F8BB00D46DDF8509083
:1033900014469B468046002800F01981B9F1000FC1
:1033A00000F01581531E3F2B00F21181012A03D139
:1033B000BBF1000F40F00B810023CDE90833B8F8D2
:1033C0001430B5EBC30F4FEAC30703D300200BB093
:1033D000BDE8F08F2B199F42D8F80C303ABF7F1B05
:1033E000FFB227461BB9D8F81030002B7AD0272D12
:1033F0004ED8C5F12806B7424FF000032CBFF6B2F5
:103400003E4600932946D8F8080008AB3246FFF73D
:1034100041FCA7EB060A35445FFA8AFAB8F8143083
:1034200003F10053053BDB000493D8F80C30039301
:103430002821039B13B1BAF1000F2CD1D8F810004A
:1034400040B1BAF1000F05D0009608AB5246691A98
:10345000FFF720FC38B2002FB8D066070AD00AABBD
:1034600003EBD401624211F8083C02F00702134159
:1034700001F8083C082C3CD9102C40F2B580202CD7
:1034800040F2B780BBF1000F00F09C80082334E0CD
:10349000BA460026C2E7049BE02B28BFE023069330
:1034A0000B44AB42059314D95A1B039800969245DE
:1034B00034BF5246D2B2691A08AB04300792FFF704
:1034C000E9FB079A1644AAEB020A1544F6B25FFA22
:1034D0008AFA049B069A05999B1A0493039B1B681E
:1034E0000393A6E70093D8F8080008AB3A462946AC
:1034F000AEE7BBF1000F13D00123B4EBC30F6CD0C8
:10350000082C12D89DF82030621E23FA02F2D5074B
:1035100006D54FF0FF3202FA04F423438DF8203031
:103520009DF8203089F8003051E7102C12D8BDF8F2
:103530002030621E23FA02F2D10706D54FF0FF3287
:1035400002FA04F42343ADF82030BDF82030A9F886
:1035500000303CE7202C0FD80899631E21FA03F3B2
:10356000DA0705D54FF0FF3202FA04F40C43089451
:10357000089BC9F800302AE7402C2BD0DDE908650C
:10358000611EC4F12102A4F1210326FA01F105FA1A
:1035900002F225FA03F311431943CB0712D5012296
:1035A000A4F12003C4F1200102FA03F322FA01F18D
:1035B000A240524243EA010363EB430332432B43ED
:1035C000CDE90823DDE90823C9E90023FFE66FF010
:1035D0000100FCE66FF00800F9E6082CA0D9102CD9
:1035E000B3D9202CEED8C3E7BBF1000FADD0022336
:1035F00083E7BBF1000FBBD004237EE730B5012A7F
:10360000144638BF0124402C85B028BF4024002533
:10361000012ACDE9025518D81B788DF808306307C8
:103620000AD004AB03EBD405624215F8083C02F063
:103630000702934005F8083C00910346224600210A
:1036400002A8FFF727FB05B030BD082AE4D9102AED
:1036500003D81B88ADF80830E1E7202A8DBFD3E9F5
:1036600000231B680293CDE90223D8E710B5CB688D
:103670001BB98B600B618B8210BD04691A681C60DA
:103680000361C38A013BC382CA60F0E703064CBFF3
:10369000C0F3C0300220704708B50246FFF7F6FFBE
:1036A000022806D15306C2F30F2001D100F0030017
:1036B00008BDC2F30740FBE72DE9F04F93B0CDE919
:1036C00003230A6804461046FFF7E0FF022814BFF0
:1036D000C2F306260026002A0D46824680F2F281B9
:1036E00012F0C04940F0EE81097B002900F0EA8128
:1036F000022803D02378B34240F0E781C2F3046389
:103700000693104602F07F030593FFF7C5FF059B64
:1037100029444FEA834848EA0A4848EA4668CE788E
:1037200000230022CDE90823F309834648EA000874
:10373000029367D0059B009302466768534608A929
:103740002046B847002800F0C381276A4FB9414698
:1037500004F10C00FFF702FB074690B96FF002007E
:1037600054E03B6998450DD03F68002FF9D14146A0
:1037700004F10C00FFF7F2FA07460028EED0236AA6
:103780003B60276297F817C006F01F08CCF3840C43
:10379000ACEB08001FFA80FE0028B8BF0EF1200035
:1037A000A8EB0C031FFA83FED7E90221B8BF00B2D1
:1037B000002B0793BEBF0EF120031BB2079352EA02
:1037C000010338D0039BDFF824E39A1A049B4FF0DF
:1037D000000C63EB010196457CEB01032BD36B7B63
:1037E00097F81AE0734519D1029B002B78D0012875
:1037F00021DC7868F8B9DFF8F0C2944570EB01037A
:1038000016D337E0276A27B96FF00C0013B0BDE874
:10381000F08F3B699845B5D03F68F4E7B2489042D5
:103820007CEB010301D30020F0E7029B002BFAD0D0
:10383000079B0F2B17DCFA7DB30002F0030203F0A5
:103840007C031343FB7539462046FFF707FB6B7B70
:10385000BB76029B3BB9FB7DC3F38402013262F36A
:103860008603FB75D0E76A7BBB7E9A42DBD1029B65
:10387000002B35D0B309022B32D0039BBB60049BD5
:10388000FB60142200210DA8FEF766F8039B0A9343
:10389000049B0B932B1D0C932B7BADF83EB0013B8F
:1038A000DBB2ADF83C30069B8DF84230059B8DF8BD
:1038B000433094F82C308DF840A083F001038DF84C
:1038C00044308DF84180A3680AA920469847FB7DC3
:1038D000C3F38403013303F01F039B02FB82A2E7BF
:1038E000FB7DC6F34012B2EBD31F40F0F480C3F36C
:1038F0008403434540F0F280029A2B7BB609002AEC
:103900004DD0F2075DD4032B40F2EB80039BBB60EC
:10391000049BFB602B7BAE1D033BDBB2324639467A
:1039200004F10C00FFF7ACFA00280CDA3946204607
:10393000FFF794FAFB7DC3F38403013303F01F0305
:103940009B02FB820AE7DDE90884AB883B834FF6E4
:10395000FF73C9F12000A9F1200228FA09F104FA45
:1039600000F0014324FA02F211431846C9B2FFF7EE
:10397000C9F909F10809B9F1400F0346E9D1B88244
:103980002A7B033AD2B23146FFF7CEF9FB7DB882EB
:10399000DA43C2F3C01262F3C713FB7543E786B97B
:1039A0002E1D013BDBB23246394604F10C00FFF715
:1039B00067FA0028BADB2A7BB88A013AD2B23146CC
:1039C000E2E7F98AC1F30901013B0429DAB25BD8C5
:1039D000281D002307F11B069A4208D910F801CBD5
:1039E00006F801C0013101330529DBB2F4D1039996
:1039F0000A9104990B91934207F11B010C9138BF76
:103A0000043379680D9134BF55FA83F300230E9384
:103A1000FB8AADF83EB0C3F309031A44069B8DF848
:103A20004230059B8DF8433094F82C30ADF83C20A3
:103A300083F001038DF8443000238DF840A08DF809
:103A400041807B602A7BB88A013A291DFFF76CF917
:103A50003B8BB882834203D1A3680AA920469847CA
:103A600020460AA9FFF702FEFB7DBA8AC3F384034E
:103A7000013303F01F039B02FB823B8B9A420CBF76
:103A800000206FF01000C1E67B68002BAFD005204E
:103A900001E01C3033461E68002EFAD1091A081DB9
:103AA0002E1D184401EB090CBCF11B0F5FFA89F3C2
:103AB0009DD89A429BD916F8013B00F8013B09F1C9
:103AC0000109EFE76FF00900A0E66FF00A009DE63C
:103AD0006FF00B009AE66FF00D0097E66FF00E00A6
:103AE00094E66FF00F0091E640420F0080841E00C4
:103AF000EFF3098305494A6B22F001024A636833F8
:103B000083F30988002383F31188704700EF00E0F6
:103B1000302080F3118862B60C4B0D4AD96821F42D
:103B2000E0610904090C0A43DA60D3F8FC20094972
:103B300042F08072C3F8FC200A6842F001020A6079
:103B40002022DA7783F82200704700BF00ED00E002
:103B50000003FA05001000E010B5302383F311884C
:103B60000E4B5B6813F4006314D0F1EE103AEFF3E0
:103B70000984683C4FF08073E361094BDB6B23667B
:103B800084F3098800F08AFB10B1064BA36110BDD5
:103B9000054BFBE783F31188F9E700BF00ED00E078
:103BA00000EF00E04306000846060008026843688C
:103BB0001143016003B1184770470000024AD368FF
:103BC00043F0C003D360704700100140024AD3683D
:103BD00043F0C003D36070470044004010B50A4C66
:103BE0000A4A2046002100F0A9FA094B094AC4E913
:103BF0009723094C094A0021204600F09FFA084902
:103C0000084BC4E9971310BD08470020BD3B0008CE
:103C100080F0FA020010014074490020CD3B0008FA
:103C20000044004040787D012A4A037C002918BFE7
:103C30000A46012B30B5C0F868220CD1264B9842B9
:103C400039D1264B596C41F010015964596E41F03D
:103C5000100159665B6EB2F904501468D0F86032F6
:103C6000D0F85C12002D03EB5403B3FBF4F3BEBF9A
:103C700023F0070503F0070343EA450394888B60AC
:103C8000D38843F040030B61138943F001034B6178
:103C900044F4045343F02C03CB6004F4A0540023F9
:103CA0000B60B4F5806F0B684B680CBF7F23FF235C
:103CB00080F8643230BD0A4B9842CCD1074B196C66
:103CC00041F400311964196E41F4003119661B6E1C
:103CD000C1E700BF1C54000808470020003802401C
:103CE000744900202DE9F041D0F85C62F768336830
:103CF000DA0504469DB20DD5302383F311884FF4C5
:103D000080610430FFF752FF6FF48073336000234B
:103D100083F31188302383F3118804F1040815F02C
:103D20002F033AD183F31188380615D5290613D508
:103D3000302383F3118804F1380000F07BF9002868
:103D40004EDA0821201DFFF731FF4FF67F733B400D
:103D5000F360002383F311887A0616D56B0614D519
:103D6000302383F31188D4E913239A420AD1236CB8
:103D700043B127F040073F041021201D3F0CFFF7FF
:103D800015FFF760002383F31188D4F86822D36805
:103D900043B3BDE8F041106918472B0714D015F064
:103DA000080F0CBF00214FF48071E80748BF41F0B5
:103DB0002001AA0748BF41F040016B0748BF41F00E
:103DC00080014046FFF7F2FEAD06736805D594F812
:103DD00064122046194000F0E1F93568ADB29EE763
:103DE0007060B6E7BDE8F08100F1604303F5614320
:103DF0000901C9B283F80013012200F01F039A40A1
:103E000043099B0003F1604303F56143C3F880213C
:103E10001A607047F8B5154682680669AA420B46D3
:103E2000816938BF8568761AB54204460BD21846B8
:103E30002A46FDF77FFDA3692B44A361A3685B1BA2
:103E4000A3602846F8BD0CD918463246FDF772FD2E
:103E5000AF1BE1683A463044FDF76CFDE3683B4434
:103E6000EBE718462A46FDF765FDE368E5E7000045
:103E700083689342F7B51546044638BF8568D0E994
:103E80000460361AB5420BD22A46FDF753FD63692A
:103E90002B446361A36828465B1BA36003B0F0BD9D
:103EA0000DD932460191FDF745FD0199E068AF1B40
:103EB0003A463144FDF73EFDE3683B44E9E72A46D4
:103EC000FDF738FDE368E4E710B50A440024C36158
:103ED000029B8460C0E90000C0E90511C160026175
:103EE000036210BD08B5D0E90532934201D1826862
:103EF00082B98268013282605A1C42611970D0E92D
:103F000004329A4224BFC3684361002100F08EFA54
:103F1000002008BD4FF0FF30FBE7000070B53023F4
:103F200004460E4683F31188A568A5B1A368A2696B
:103F3000013BA360531CA36115782269934224BFFF
:103F4000E368A361E3690BB120469847002383F33C
:103F50001188284607E03146204600F057FA00282D
:103F6000E2DA85F3118870BD2DE9F74F04460E465D
:103F700017469846D0F81C904FF0300A8AF3118803
:103F80004FF0000B154665B12A4631462046FFF733
:103F900041FF034660B94146204600F037FA002849
:103FA000F1D0002383F31188781B03B0BDE8F08FB4
:103FB000B9F1000F03D001902046C847019B8BF355
:103FC0001188ED1A1E448AF31188DCE7C0E9051157
:103FD000C160C3611144009B8260C0E900000161BF
:103FE00003627047F8B504460D461646302383F346
:103FF0001188A768A7B1A368013BA36063695A1C35
:1040000062611D70D4E904329A4224BFE36863619F
:10401000E3690BB120469847002080F3118807E040
:104020003146204600F0F2F90028E2DA87F31188E1
:10403000F8BD0000D0E905239A4210B501D182688D
:104040007AB98268013282605A1C82611C780369E5
:104050009A4224BFC3688361002100F0E7F920463B
:1040600010BD4FF0FF30FBE72DE9F74F04460E4639
:1040700017469846D0F81C904FF0300A8AF3118802
:104080004FF0000B154665B12A4631462046FFF732
:10409000EFFE034660B94146204600F0B7F900281C
:1040A000F1D0002383F31188781B03B0BDE8F08FB3
:1040B000B9F1000F03D001902046C847019B8BF354
:1040C0001188ED1A1E448AF31188DCE70268436800
:1040D0001143016003B11847704700001430FFF727
:1040E00043BF00004FF0FF331430FFF73DBF000027
:1040F0003830FFF7B9BF00004FF0FF333830FFF71B
:10410000B3BF00001430FFF709BF00004FF0FF31CC
:104110001430FFF703BF00003830FFF763BF000023
:104120004FF0FF323830FFF75DBF0000012914BFA8
:104130006FF0130000207047FFF750BD37B51546EC
:104140000E4A026000224260C0E9022201220446B7
:1041500002740B46009000F15C014FF48072143041
:10416000FFF7B2FE00942B464FF4807204F5AE7157
:1041700004F13800FFF72AFF03B030BD30540008C7
:1041800010B53023044683F31188FFF74DFD022359
:104190002374002080F3118810BD000038B5C36976
:1041A00004460D461BB904210844FFF78FFF29463A
:1041B00004F11400FFF796FE002806DA201D4FF4E4
:1041C0000061BDE83840FFF781BF38BD00230375AB
:1041D000826803691B6899689142FBD25A68036040
:1041E000426010605860704700230375826803695D
:1041F0001B6899689142FBD85A680360426010605E
:104200005860704708B50846302383F311880B7D4A
:10421000032B05D0042B0DD02BB983F3118808BDD7
:104220008B6900221A604FF0FF338361FFF7CEFFE6
:104230000023F2E7D1E9003213605A60F3E700008F
:10424000FFF7C4BF054BD9680875186802681A6083
:10425000536001220275D860FCF7DEB9E04B002004
:1042600030B50C4BDD684B1C87B004460FD02B4695
:10427000094A684600F06CF92046FFF7E3FF009B0F
:1042800013B1684600F06EF9A86907B030BDFFF7BA
:10429000D9FFF9E7E04B002005420008044B1A68FB
:1042A000DB6890689B68984294BF002001207047AB
:1042B000E04B0020084B10B51C68D86822681A60D3
:1042C000536001222275DC60FFF78EFF0146204615
:1042D000BDE81040FCF7A0B9E04B0020044B1A6881
:1042E000DB6892689B689A4201D9FFF7E3BF704789
:1042F000E04B002038B5074C07490848012300254A
:104300002370656000F052FC0223237085F311884E
:1043100038BD00BF484E00205C540008E04B002030
:1043200008B572B6044B186500F0FEFA00F0B2FB57
:10433000024B03221A70FEE7E04B0020484E00209B
:1043400000F046B9EFF3118020B9EFF30583302276
:1043500082F311887047000010B530B9EFF305847F
:10436000C4F3080414B180F3118810BDFFF7B6FF41
:1043700084F31188F9E700008B60022308618B82C7
:10438000084670478368A3F1840243F8142C02693D
:1043900043F8442C426943F8402C094A43F8242C42
:1043A000C26843F8182C022203F80C2C002203F8F0
:1043B0000B2C044A43F8102CA3F12000704700BFD7
:1043C00031060008E04B002008B5FFF7DBFFBDE831
:1043D0000840FFF735BF0000024BDB6898610F20F3
:1043E000FFF730BFE04B0020302383F31188FFF745
:1043F000F3BF000008B50146302383F3118808207D
:10440000FFF72EFF002383F3118808BD064BDB68FE
:1044100039B1426818605A60136043600420FFF7A6
:104420001FBF4FF0FF307047E04B002003689842F9
:1044300006D01A680260506099611846FFF700BF05
:104440007047000010B503689C68A2420CD85C68F5
:104450008A600B604C602160596099688A1A9A6082
:104460004FF0FF33836010BD1B68121BECE70000A8
:104470000A2938BF0A2170B504460D460A2660197C
:1044800000F08CFB00F074FB041BA54203D8751CE4
:104490002E460446F3E70A2E04D9BDE870400120F9
:1044A00000F0C4BB70BD0000F8B5144B0D46D961D7
:1044B00003F1100141600A2A1969826038BF0A229B
:1044C000016048601861A818144600F057FB0A27DD
:1044D00000F04EFB431BA342064606D37C1C281962
:1044E00000F05CFB27463546F2E70A2F04D9BDE809
:1044F000F840012000F09ABBF8BD00BFE04B00205F
:10450000F8B506460D4600F033FB0F4A134653F844
:10451000107F9F4206D12A4601463046BDE8F8404A
:10452000FFF7C2BFD169BB68441A2C1928BF2C46BB
:10453000A34202D92946FFF79BFF22463146034892
:10454000BDE8F840FFF77EBFE04B0020F04B0020B5
:1045500010B4C0E9032300235DF8044B4361FFF767
:10456000CFBF000010B5194C236998420DD0D0E997
:104570000032816813605A609A680A449A60002386
:1045800003604FF0FF33A36110BD2346026843F878
:10459000102F53600022026022699A4203D1BDE8C5
:1045A000104000F0F5BA936881680B44936000F006
:1045B000DFFA2269E1699268441AA242E4D91144FF
:1045C000BDE81040091AFFF753BF00BFE04B0020C1
:1045D0002DE9F047DFF8BC8008F110072C4ED8F821
:1045E000105000F0C5FAD8F81C40AA68031B9A4284
:1045F0003ED81444D5E900324FF00009C8F81C40F9
:1046000013605A60C5F80090D8F81030B34201D159
:1046100000F0BEFA89F31188D5E90331284698479E
:10462000302383F311886B69002BD8D000F0A0FAF7
:104630006A69A0EB04094A4582460DD2022000F0C7
:10464000F5FA0022D8F81030B34208D15146284676
:10465000BDE8F047FFF728BF121A2244F2E712EB39
:10466000090938BF4A4629463846FFF7EBFEB5E749
:10467000D8F81030B34208D01444211AC8F81C00EE
:10468000A960BDE8F047FFF7F3BEBDE8F08700BFC3
:10469000F04B0020E04B002000207047FEE70000B8
:1046A000704700004FF0FF3070470000BFF34F8F9E
:1046B000024AD368DB03FCD4704700BF003C0240D1
:1046C00008B5094B1B7873B9FFF7F0FF074B1A6960
:1046D000002ABFBF064A5A6002F188325A601A683F
:1046E00022F480621A6008BD504E0020003C024057
:1046F0002301674508B50B4B1B7893B9FFF7D6FF2D
:10470000094B1A6942F000421A611A6842F4805259
:104710001A601A6822F480521A601A6842F48062A1
:104720001A6008BD504E0020003C02400B28F0B536
:1047300016D80C4C0C4923787BB90C4D0E460C2333
:104740004FF0006255F8047B46F8042B013B13F050
:10475000FF033A44F6D10123237051F82000F0BD45
:104760000020FCE7844E0020544E002068540008CE
:10477000014B53F820007047685400080C20704724
:104780000B2810B5044601D9002010BDFFF7CEFF5D
:10479000064B53F824301844C21A0BB90120F4E731
:1047A00012680132F0D1043BF6E700BF68540008FC
:1047B0000B2838B5044628D8FFF7C4FDFFF776FF6D
:1047C000FFF77EFF124AF323D360E300DBB243F42A
:1047D000007343F002031361136943F480331361E0
:1047E00005462046FFF762FFFFF7A0FF094B53F88D
:1047F000241000F04BF92846FFF77CFFFFF7ACFDD3
:104800002046BDE83840FFF7BBBF002038BD00BFE1
:10481000003C02406854000812F001032DE9F04109
:1048200005460E4614464BD18218B2F1016F61D88D
:10483000314B1B6813F001035CD0304FFFF782FD52
:10484000FFF73EFFF323FB60FFF730FF314640F2F6
:104850000128032C18D824F00104284E0C446D1AAA
:1048600040F20118A142336905EB01072AD123F078
:1048700001033361FFF73EFFFFF76EFD0120BDE846
:10488000F081043C0435E4E7AB07E4D13B6923F451
:1048900040733B613B6943EA08033B6151F8046B99
:1048A0002E60BFF34F8FFFF701FF2B689E42E8D0C9
:1048B0003B6923F001033B61FFF71CFFFFF74CFD51
:1048C0000020DCE723F440733361336943EA0803D3
:1048D00033610B883B80BFF34F8FFFF7E7FE3F88C4
:1048E00031F8023BBFB2BB42BCD0336923F00103B5
:1048F0003361E1E71846C2E700380240003C02405D
:10490000084908B50B7828B11BB9FFF7D9FE012378
:104910000B7008BD002BFCD0BDE808400870FFF705
:10492000E9BE00BF504E00204FF480214FF00050F0
:1049300000F0AEB80846114600F050BC012000F06F
:104940004DBC0000084600F067BC000070B582B0A6
:10495000FFF7F8FC0E4E054600F00AF93268904267
:1049600037BF0C4A0B49516814682EBFD1E900418A
:10497000013151600419034641F1000128460191BB
:104980003360FFF7E9FC0199204602B070BD00BF1B
:10499000884E0020904E002070B582B0FFF7D2FC08
:1049A000104E054600F0E4F83268904237BF0E4AD8
:1049B0000D49516814682EBFD1E9004101315160A1
:1049C000041941F100010346284601913360FFF7C5
:1049D000C3FC01994FF47A7200232046FBF708FCD0
:1049E00002B070BD884E0020904E002010B50244E9
:1049F000064BD2B2904200D110BD441C00B253F815
:104A0000200041F8040BE0B2F4E700BF502800405A
:104A10000F4B30B51C6F240407D41C6F44F4007492
:104A20001C671C6F44F400441C670A4C236843F461
:104A3000807323600244084BD2B2904200D130BD53
:104A4000441C00B251F8045B43F82050E0B2F4E794
:104A500000380240007000405028004007B5012295
:104A600001A90020FFF7C2FF019803B05DF804FB25
:104A700013B50446FFF7F2FFA04205D0012201A9B9
:104A800000200194FFF7C4FF02B010BD7047000082
:104A90007047000070470000074B45F255521A60FE
:104AA00002225A6040F6FF729A604CF6CC421A60BD
:104AB000024B01221A707047003000409C4E0020CB
:104AC000034B1B781BB1034B4AF6AA221A607047AE
:104AD0009C4E002000300040034B1A681AB9034A6C
:104AE000D2F874281A607047984E002000300240B7
:104AF000024B4FF08072C3F87428704700300240B8
:104B000008B5FFF7E9FF024B1868C0F3407008BD15
:104B1000984E002008B5FFF7DFFF024B1868C0F37E
:104B2000007008BD984E002070470000FEE70000AE
:104B30000A4B0B480B4A90420BD30B4BDA1C121A50
:104B4000C11E22F003028B4238BF00220021FCF775
:104B500003BF53F8041B40F8041BECE71C56000885
:104B6000284F0020284F0020284F002000F0D0B808
:104B7000014B586A704700BF000C0040034B0022F5
:104B800058631A610222DA60704700BF000C0040CF
:104B9000014B0022DA607047000C0040014B586363
:104BA000704700BF000C0040FEE7000070B51B4BD3
:104BB00001630025044686B0586085620E46FEF704
:104BC000A7FF04F11003C4E904334FF0FF33C4E935
:104BD0000635C4E90044A560E562FFF7C9FF2B462E
:104BE0000246C4E9082304F134010D4A25658023F7
:104BF0002046FFF7C1FB0123E0600A4A03750092DB
:104C000072680192B268CDE90223074B6846CDE98C
:104C10000435FFF7D9FB06B070BD00BF484E002039
:104C2000985400089D540008A94B0008024AD36A12
:104C30001843D062704700BFE04B00204B684360D0
:104C40008B688360CB68C3600B6943614B69036207
:104C50008B6943620B6803607047000008B5234B03
:104C600023481A6942F0FF021A611A6922F0FF0212
:104C70001A611A691A6B42F0FF021A631A6D42F048
:104C8000FF021A651B4A1B6D1146FFF7D7FF02F1A1
:104C90001C0100F58060FFF7D1FF02F1380100F53B
:104CA0008060FFF7CBFF02F1540100F58060FFF751
:104CB000C5FF02F1700100F58060FFF7BFFF02F150
:104CC0008C0100F58060FFF7B9FF02F1A80100F543
:104CD0008060FFF7B3FF02F1C40100F58060FFF7C9
:104CE000ADFFBDE8084000F08FB800BF00380240BB
:104CF00000000240A454000808B500F029FAFFF7AC
:104D0000F9FABDE80840FFF7E7BE00007047000071
:104D10000E4B1A6C42F008021A641A6E42F0080236
:104D20001A660B4A1B6E936843F008039360094BA5
:104D300031229A624FF0FF32DA6200229A615A639E
:104D4000DA605A6001225A611A60704700380240E6
:104D5000002004E0000C0040094A08B51169D3683E
:104D60000B40D9B2C9439B07116107D5302383F3A8
:104D70001188FFF7E5FA002383F3118808BD00BF0F
:104D8000000C00401E4B1A6962F0FF021A611A699A
:104D9000D2B21A614FF0FF301A695A695861002186
:104DA0005A6959615A691A6A62F080521A621A6A1B
:104DB00002F080521A621A6A5A6A58625A6A596232
:104DC0005A6A1A6C42F080521A641A6E42F080528B
:104DD0001A661A6E0B4A106840F480701060186FE3
:104DE00000F44070B0F5007F1EBF4FF480301867AC
:104DF0001967536823F40073536000F07DB900BF56
:104E000000380240007000403B4B3C4A1A643C4A68
:104E10004FF4404111601A6842F001021A601A68AA
:104E20009007FCD59A6822F003029A60324B9A6888
:104E300012F00C02FBD1196801F0F90119609A60B7
:104E40001A6842F480321A601A689103FCD55A6FCE
:104E500042F001025A67284B5A6F9207FCD5294A43
:104E60005A601A6842F080721A60254A53685804E2
:104E7000FCD5214B1A689101FCD5234AC3F8842044
:104E80001A6842F080621A601A681201FCD51F4A43
:104E90009A600322C3F88C204FF00062C3F894207C
:104EA0001B4B1A681B4B9A421B4B21D11B4A1168A2
:104EB0001B4A91421CD140F203121A60164A136831
:104EC00003F00F03032BFAD10B4B9A6842F0020256
:104ED0009A609A6802F00C02082AFAD15A6C42F4DD
:104EE00080425A645A6E42F480425A665B6E704742
:104EF00040F20372E1E700BF0038024000040010F6
:104F000000700040041940020830002400948838E2
:104F1000002004E011640020003C024000ED00E0AD
:104F200041C20F41074A08B5536903F001035361B9
:104F300023B1054A13680BB150689847BDE8084093
:104F4000FEF70ABE003C0140A04E0020074A08B50B
:104F5000536903F00203536123B1054A93680BB10F
:104F6000D0689847BDE80840FEF7F6BD003C014018
:104F7000A04E0020074A08B5536903F004035361AB
:104F800023B1054A13690BB150699847BDE8084041
:104F9000FEF7E2BD003C0140A04E0020074A08B5E4
:104FA000536903F00803536123B1054A93690BB1B8
:104FB000D0699847BDE80840FEF7CEBD003C0140EF
:104FC000A04E0020074A08B5536903F0100353614F
:104FD00023B1054A136A0BB1506A9847BDE80840EF
:104FE000FEF7BABD003C0140A04E0020164B10B5A4
:104FF0005C6904F478725A61A30604D5134A936A73
:105000000BB1D06A9847600604D5104A136B0BB1F8
:10501000506B9847210604D50C4A936B0BB1D06BAB
:105020009847E20504D5094A136C0BB1506C9847B8
:10503000A30504D5054A936C0BB1D06C9847BDE825
:105040001040FEF789BD00BF003C0140A04E00208B
:10505000194B10B55C6904F47C425A61620504D5B1
:10506000164A136D0BB1506D9847230504D5134AAA
:10507000936D0BB1D06D9847E00404D50F4A136EC1
:105080000BB1506E9847A10404D50C4A936E0BB136
:10509000D06E9847620404D5084A136F0BB1506F65
:1050A0009847230404D5054A936F0BB1D06F9847F6
:1050B000BDE81040FEF750BD003C0140A04E00206E
:1050C00008B50348FEF70EFEBDE80840FEF744BDF4
:1050D0000847002008B50348FEF704FEBDE8084075
:1050E000FEF73ABD7449002008B5FFF735FEBDE86C
:1050F0000840FEF731BD0000062108B50846FEF75E
:1051000073FE06210720FEF76FFE06210820FEF73A
:105110006BFE06210920FEF767FE06210A20FEF736
:1051200063FE06211720FEF75FFE06212820FEF70A
:105130005BFE07213220FEF757FE0C212520FEF7EB
:1051400053FEBDE808400C212620FEF74DBE0000AE
:1051500008B5FFF717FE00F009F8FEF7EDFFFFF7BF
:10516000D5FDBDE80840FFF701BD00000023054A5A
:1051700019460133102BC2E9001102F10802F8D1DF
:10518000704700BFA04E00200B460146184600F0B5
:105190002DB8000000F040B8012838BF012010B53C
:1051A0000446204600F030F830B900F007F808B99E
:1051B00000F00CF88047F4E710BD0000024B1868BF
:1051C000BFF35B8F704700BF204F002008B506205B
:1051D00000F084F80120FFF761FA0000024B0A4654
:1051E00001461868FFF7A6BB2823002010B5054C20
:1051F00013462CB10A4601460220AFF3008010BDD1
:105200002046FCE700000000024B01461868FFF74B
:1052100095BB00BF28230020024B01461868FFF70A
:1052200091BB00BF2823002010B5013902449042F1
:1052300001D1002005E0037811F8014FA34201D00D
:10524000181B10BD0130F2E72DE9F041A3B1C91AD6
:1052500017780144044603F1FF3C8C42204601D9F3
:10526000002009E00578BD4204F10104F5D10CEB02
:105270000405D618A54201D1BDE8F08115F8018DCD
:1052800016F801EDF045F5D0E7E700001F2938B525
:1052900004460D4604D9162303604FF0FF3038BD95
:1052A000426C12B152F821304BB9204600F030F870
:1052B0002A4601462046BDE8384000F017B8012BC9
:1052C0000AD0591C03D1162303600120E7E700240C
:1052D00042F82540284698470020E0E7024B014667
:1052E0001868FFF7D3BF00BF2823002038B5074D4B
:1052F00000230446084611462B60FFF7D3F9431CF0
:1053000002D12B6803B1236038BD00BF244F0020B9
:10531000FFF7C2B9034611F8012B03F8012B002A4D
:10532000F9D170476F72672E6172647570696C6F26
:10533000742E41524B5F43414E4E4F444500000096
:1053400053544D3332463F3F3F0053544D33324662
:105350003430780053544D3332463432780053544D
:105360004D333246343436585800000001203300A3
:105370000010410001105A000310590007103100BD
:105380000000000040530008130400004A530008C6
:105390001904000054530008210400005E53000863
:1053A00040A2E4F1646891060041A3E5F2656992C8
:1053B000070000004261642043414E496661636515
:1053C00020696E6465782E00800000000080000077
:1053D00000008000000000000000000061200008C4
:1053E00049280008A927000871200008A520000806
:1053F000A1220008752000088520000879200008F7
:10540000812000087D200008C921000889200008AB
:10541000152B0008992000089D2100080096000027
:10542000000000000000000000000000000000007C
:1054300000000000F9400008E54000082141000894
:105440000D4100081941000805410008F14000081D
:10545000DD4000082D41000863300000585400086A
:10546000384C0020484E0020004000000040000062
:1054700000400000004000000000010000000200A9
:105480000000020000000200000002000000020014
:1054900000000200000002006D61696E0069646C2A
:1054A00065000000A00195AA00070000AAAAAAAA08
:1054B00050010064FFF900000077000000900970BF
:1054C0008000000100000000AAAAAAAA4000000172
:1054D000FFFF00000070000000000000000000500E
:1054E00000000000AAAAAA5A00000000FF3F000026
:1054F00000000000000000000000000000000000AC
:10550000AAAAAAAA00000000FFFF000000000000F5
:10551000000000000000000000000000AAAAAAAAE3
:1055200000000000FFFF000000000000000000007D
:105530000000000000000000AAAAAAAA00000000C3
:10554000FFFF00000000000000000000000000005D
:1055500000000000AAAAAAAA00000000FFFF0000A5
:10556000000000000000000000000000000000003B
:105570000A0000000000000003000000000000001E
:10558000000000009CACFF7F010000000000000054
:10559000530000000000000000000F0000000000A9
:1055A00040420F00FE2A0100D2040000FF0000006C
:1055B00008470020744900202C2300200000000030
:1055C00000000000000000000000000000000000DB
:1055D00000000000000000000000000000000000CB
:1055E00000000000000000000000000000000000BB
:1055F00000000000000000000000000000000000AB
:10560000000000000000000000000000000000009A
:0C5610000000000000000000000000008E
:00000001FF
